 popframe008

 Timestamp is e2c8c2e9 (reproducible build file hash)

 Preferred load address is 0000000180000000

 Start         Length     Name                   Class
 0001:00000000 00002ff0H .text$mn                CODE
 0001:00002ff0 00000036H .text$mn$00             CODE
 0001:00003026 00000092H .text$x                 CODE
 0002:00000000 00000198H .idata$5                DATA
 0002:00000198 00000038H .00cfg                  DATA
 0002:000001d0 00000008H .CRT$XCA                DATA
 0002:000001d8 00000008H .CRT$XCZ                DATA
 0002:000001e0 00000008H .CRT$XIA                DATA
 0002:000001e8 00000008H .CRT$XIC                DATA
 0002:000001f0 00000008H .CRT$XIZ                DATA
 0002:000001f8 00000008H .CRT$XLA                DATA
 0002:00000200 00000008H .CRT$XLZ                DATA
 0002:00000208 00000008H .CRT$XPA                DATA
 0002:00000210 00000008H .CRT$XPZ                DATA
 0002:00000218 00000008H .CRT$XTA                DATA
 0002:00000220 00000010H .CRT$XTZ                DATA
 0002:00000228 00000000H .gehcont$y              DATA
 0002:00000228 00000000H .gfids$y                DATA
 0002:00000230 00001ed0H .rdata                  DATA
 0002:00002100 00000000H .rdata$CastGuardVftablesA DATA
 0002:00002100 00000000H .rdata$CastGuardVftablesC DATA
 0002:00002100 00000028H .rdata$T                DATA
 0002:00002128 000000b0H .rdata$voltmd           DATA
 0002:000021d8 00000318H .rdata$zzzdbg           DATA
 0002:000024f0 00000008H .rtc$IAA                DATA
 0002:000024f8 00000008H .rtc$IZZ                DATA
 0002:00002500 00000008H .rtc$TAA                DATA
 0002:00002508 00000008H .rtc$TZZ                DATA
 0002:00002510 00000004H .tls                    DATA
 0002:00002514 00000004H .tls$                   DATA
 0002:00002518 00000008H .tls$ZZZ                DATA
 0002:00002520 00000300H .xdata                  DATA
 0002:00002820 000003d0H .edata                  DATA
 0002:00002bf0 00000064H .idata$2                DATA
 0002:00002c54 00000014H .idata$3                DATA
 0002:00002c68 00000198H .idata$4                DATA
 0002:00002e00 0000041eH .idata$6                DATA
 0003:00000000 00000100H .data                   DATA
 0003:00000100 0001b398H .bss                    DATA
 0004:00000000 0000039cH .pdata                  DATA

  Address         Publics by Value              Rva+Base               Lib:Object

 0000:00000000       __AbsoluteZero             0000000000000000     <absolute>
 0000:00000000       ___safe_se_handler_count   0000000000000000     <absolute>
 0000:00000000       ___safe_se_handler_table   0000000000000000     <absolute>
 0000:00000000       __arm64x_extra_rfe_table   0000000000000000     <absolute>
 0000:00000000       __arm64x_extra_rfe_table_size 0000000000000000     <absolute>
 0000:00000000       __arm64x_native_entrypoint 0000000000000000     <absolute>
 0000:00000000       __arm64x_redirection_metadata 0000000000000000     <absolute>
 0000:00000000       __arm64x_redirection_metadata_count 0000000000000000     <absolute>
 0000:00000000       __dynamic_value_reloc_table 0000000000000000     <absolute>
 0000:00000000       __enclave_config           0000000000000000     <absolute>
 0000:00000000       __guard_check_icall_a64n_fptr 0000000000000000     <absolute>
 0000:00000000       __guard_eh_cont_count      0000000000000000     <absolute>
 0000:00000000       __guard_eh_cont_table      0000000000000000     <absolute>
 0000:00000000       __guard_fids_count         0000000000000000     <absolute>
 0000:00000000       __guard_fids_table         0000000000000000     <absolute>
 0000:00000000       __guard_iat_count          0000000000000000     <absolute>
 0000:00000000       __guard_iat_table          0000000000000000     <absolute>
 0000:00000000       __guard_longjmp_count      0000000000000000     <absolute>
 0000:00000000       __guard_longjmp_table      0000000000000000     <absolute>
 0000:00000000       __hybrid_auxiliary_iat     0000000000000000     <absolute>
 0000:00000000       __hybrid_auxiliary_iat_copy 0000000000000000     <absolute>
 0000:00000000       __hybrid_code_map          0000000000000000     <absolute>
 0000:00000000       __hybrid_code_map_count    0000000000000000     <absolute>
 0000:00000000       __x64_code_ranges_to_entry_points 0000000000000000     <absolute>
 0000:00000000       __x64_code_ranges_to_entry_points_count 0000000000000000     <absolute>
 0000:00000100       __guard_flags              0000000000000100     <absolute>
 0000:00000000       __ImageBase                0000000180000000     <linker-defined>
 0001:00000000       ?NewObject@JNIEnv_@@QEAAPEAV_jobject@@PEAV_jclass@@PEAU_jmethodID@@ZZ 0000000180001000 f i libpopframe008.obj
 0001:00000024       ?SetEventNotificationMode@_jvmtiEnv@@QEAA?AW4jvmtiError@@W4jvmtiEventMode@@W4jvmtiEvent@@PEAV_jobject@@ZZ 0000000180001024 f i libpopframe008.obj
 0001:0000002c       ?TranslateError@@YAPEBDW4jvmtiError@@@Z 000000018000102c f   libpopframe008.obj
 0001:000002e4       ?nsk_jni_check_exception@@YAHPEAUJNIEnv_@@QEBDH@Z 00000001800012e4 f   libpopframe008.obj
 0001:00000428       ?nsk_jni_lverify@@YAHHPEAUJNIEnv_@@HQEBDH1ZZ 0000000180001428 f   libpopframe008.obj
 0001:000004c8       Agent_Initialize           00000001800014c8 f   libpopframe008.obj
 0001:00000668       Agent_OnAttach             0000000180001668 f   libpopframe008.obj
 0001:00000668       Agent_OnLoad               0000000180001668 f   libpopframe008.obj
 0001:00000670       Breakpoint                 0000000180001670 f   libpopframe008.obj
 0001:00000784       Java_nsk_jvmti_PopFrame_popframe008_getReady 0000000180001784 f   libpopframe008.obj
 0001:000008d4       Java_nsk_jvmti_PopFrame_popframe008_getRes 00000001800018d4 f   libpopframe008.obj
 0001:00000910       Java_nsk_jvmti_unit_FollowReferences_FollowRefObjects_addRefToVerify 0000000180001910 f   libpopframe008.obj
 0001:00000acc       Java_nsk_jvmti_unit_FollowReferences_FollowRefObjects_getTag 0000000180001acc f   libpopframe008.obj
 0001:00000b88       Java_nsk_jvmti_unit_FollowReferences_FollowRefObjects_resetRefsToVerify 0000000180001b88 f   libpopframe008.obj
 0001:00000b90       Java_nsk_jvmti_unit_FollowReferences_FollowRefObjects_resetTags 0000000180001b90 f   libpopframe008.obj
 0001:00000bd4       Java_nsk_jvmti_unit_FollowReferences_FollowRefObjects_setTag 0000000180001bd4 f   libpopframe008.obj
 0001:00000e20       Java_nsk_share_jvmti_ArgumentHandler_getAgentOptionsString 0000000180001e20 f   libpopframe008.obj
 0001:00000ecc       Java_nsk_share_jvmti_DebugeeClass_checkStatus 0000000180001ecc f   libpopframe008.obj
 0001:00000f54       Java_nsk_share_jvmti_DebugeeClass_resetAgentData 0000000180001f54 f   libpopframe008.obj
 0001:00000fb4       Java_nsk_share_jvmti_RedefineAgent_agentStatus 0000000180001fb4 f   libpopframe008.obj
 0001:00000fc0       Java_nsk_share_jvmti_RedefineAgent_isRedefined 0000000180001fc0 f   libpopframe008.obj
 0001:00000fcc       Java_nsk_share_jvmti_RedefineAgent_redefineAttempted 0000000180001fcc f   libpopframe008.obj
 0001:00000fd8       MA_checkStatus             0000000180001fd8 f   libpopframe008.obj
 0001:0000107c       SingleStep                 000000018000207c f   libpopframe008.obj
 0001:00001144       __local_stdio_printf_options 0000000180002144 f i libpopframe008.obj
 0001:00001314       check                      0000000180002314 f   libpopframe008.obj
 0001:00001574       exitOnError                0000000180002574 f   libpopframe008.obj
 0001:00001628       fprintf                    0000000180002628 f i libpopframe008.obj
 0001:0000166c       nsk_jvmti_lverify          000000018000266c f   libpopframe008.obj
 0001:0000175c       nsk_jvmti_resetAgentData   000000018000275c f   libpopframe008.obj
 0001:000017d0       nsk_lcomplain              00000001800027d0 f   libpopframe008.obj
 0001:000017f0       nsk_ldisplay               00000001800027f0 f   libpopframe008.obj
 0001:00001810       nsk_ltrace                 0000000180002810 f   libpopframe008.obj
 0001:00001830       nsk_lvcomplain             0000000180002830 f   libpopframe008.obj
 0001:000019e8       nsk_lvdisplay              00000001800029e8 f   libpopframe008.obj
 0001:00001a34       nsk_lverify                0000000180002a34 f   libpopframe008.obj
 0001:00001a90       nsk_lvtrace                0000000180002a90 f   libpopframe008.obj
 0001:00001af0       nsk_printf                 0000000180002af0 f   libpopframe008.obj
 0001:00001b18       nsk_vprintf                0000000180002b18 f   libpopframe008.obj
 0001:00001bcc       printf                     0000000180002bcc f i libpopframe008.obj
 0001:000020cc       __raise_securityfailure    00000001800030cc f   MSVCRT:gs_report.obj
 0001:00002100       __report_gsfailure         0000000180003100 f   MSVCRT:gs_report.obj
 0001:00002340       __GSHandlerCheck           0000000180003340 f   MSVCRT:gshandler.obj
 0001:00002360       __GSHandlerCheckCommon     0000000180003360 f   MSVCRT:gshandler.obj
 0001:000023d0       __security_check_cookie    00000001800033d0 f   MSVCRT:amdsecgs.obj
 0001:00002710       _DllMainCRTStartup         0000000180003710 f   MSVCRT:dll_dllmain.obj
 0001:00002750       __scrt_acquire_startup_lock 0000000180003750 f   MSVCRT:utility.obj
 0001:0000278c       __scrt_dllmain_after_initialize_c 000000018000378c f   MSVCRT:utility.obj
 0001:000027c0       __scrt_dllmain_before_initialize_c 00000001800037c0 f   MSVCRT:utility.obj
 0001:000027d8       __scrt_dllmain_crt_thread_attach 00000001800037d8 f   MSVCRT:utility.obj
 0001:00002800       __scrt_dllmain_crt_thread_detach 0000000180003800 f   MSVCRT:utility.obj
 0001:00002818       __scrt_dllmain_exception_filter 0000000180003818 f   MSVCRT:utility.obj
 0001:00002878       __scrt_dllmain_uninitialize_c 0000000180003878 f   MSVCRT:utility.obj
 0001:000028a8       __scrt_dllmain_uninitialize_critical 00000001800038a8 f   MSVCRT:utility.obj
 0001:000028bc       __scrt_initialize_crt      00000001800038bc f   MSVCRT:utility.obj
 0001:00002908       __scrt_initialize_onexit_tables 0000000180003908 f   MSVCRT:utility.obj
 0001:00002994       __scrt_is_nonwritable_in_current_image 0000000180003994 f   MSVCRT:utility.obj
 0001:00002a2c       __scrt_release_startup_lock 0000000180003a2c f   MSVCRT:utility.obj
 0001:00002a50       __scrt_uninitialize_crt    0000000180003a50 f   MSVCRT:utility.obj
 0001:00002a7c       _onexit                    0000000180003a7c f   MSVCRT:utility.obj
 0001:00002ab8       atexit                     0000000180003ab8 f   MSVCRT:utility.obj
 0001:00002ad0       __crt_debugger_hook        0000000180003ad0 f   MSVCRT:utility_desktop.obj
 0001:00002ad8       __scrt_fastfail            0000000180003ad8 f   MSVCRT:utility_desktop.obj
 0001:00002c24       _guard_check_icall_nop     0000000180003c24 f i MSVCRT:guard_support.obj
 0001:00002c28       __security_init_cookie     0000000180003c28 f   MSVCRT:gs_support.obj
 0001:00002cd4       DllMain                    0000000180003cd4 f   MSVCRT:dll_dllmain_stub.obj
 0001:00002cf8       ?__scrt_initialize_type_info@@YAXXZ 0000000180003cf8 f   MSVCRT:tncleanup.obj
 0001:00002d08       ?__scrt_uninitialize_type_info@@YAXXZ 0000000180003d08 f   MSVCRT:tncleanup.obj
 0001:00002d14       __local_stdio_scanf_options 0000000180003d14 f i MSVCRT:default_local_stdio_options.obj
 0001:00002d1c       __scrt_initialize_default_local_stdio_options 0000000180003d1c f   MSVCRT:default_local_stdio_options.obj
 0001:00002d38       __scrt_get_dyn_tls_init_callback 0000000180003d38 f   MSVCRT:dyn_tls_init.obj
 0001:00002d40       _RTC_Initialize            0000000180003d40 f   MSVCRT:initsect.obj
 0001:00002d7c       _RTC_Terminate             0000000180003d7c f   MSVCRT:initsect.obj
 0001:00002db8       __isa_available_init       0000000180003db8 f   MSVCRT:cpu_disp.obj
 0001:00002f64       _get_startup_argv_mode     0000000180003f64 f   MSVCRT:argv_mode.obj
 0001:00002f6c       __scrt_is_ucrt_dll_in_use  0000000180003f6c f   MSVCRT:ucrt_detection.obj
 0001:00002f80       memcpy                     0000000180003f80 f   vcruntime:VCRUNTIME140.dll
 0001:00002f86       memset                     0000000180003f86 f   vcruntime:VCRUNTIME140.dll
 0001:00002f8c       strchr                     0000000180003f8c f   vcruntime:VCRUNTIME140.dll
 0001:00002f92       __C_specific_handler       0000000180003f92 f   vcruntime:VCRUNTIME140.dll
 0001:00002f98       __std_type_info_destroy_list 0000000180003f98 f   vcruntime:VCRUNTIME140.dll
 0001:00002f9e       strcmp                     0000000180003f9e f   ucrt:api-ms-win-crt-string-l1-1-0.dll
 0001:00002fa4       strlen                     0000000180003fa4 f   ucrt:api-ms-win-crt-string-l1-1-0.dll
 0001:00002faa       _initterm                  0000000180003faa f   ucrt:api-ms-win-crt-runtime-l1-1-0.dll
 0001:00002fb0       _initterm_e                0000000180003fb0 f   ucrt:api-ms-win-crt-runtime-l1-1-0.dll
 0001:00002fb6       _seh_filter_dll            0000000180003fb6 f   ucrt:api-ms-win-crt-runtime-l1-1-0.dll
 0001:00002fbc       _configure_narrow_argv     0000000180003fbc f   ucrt:api-ms-win-crt-runtime-l1-1-0.dll
 0001:00002fc2       _initialize_narrow_environment 0000000180003fc2 f   ucrt:api-ms-win-crt-runtime-l1-1-0.dll
 0001:00002fc8       _initialize_onexit_table   0000000180003fc8 f   ucrt:api-ms-win-crt-runtime-l1-1-0.dll
 0001:00002fce       _register_onexit_function  0000000180003fce f   ucrt:api-ms-win-crt-runtime-l1-1-0.dll
 0001:00002fd4       _execute_onexit_table      0000000180003fd4 f   ucrt:api-ms-win-crt-runtime-l1-1-0.dll
 0001:00002fda       _crt_atexit                0000000180003fda f   ucrt:api-ms-win-crt-runtime-l1-1-0.dll
 0001:00002fe0       _cexit                     0000000180003fe0 f   ucrt:api-ms-win-crt-runtime-l1-1-0.dll
 0001:00002fe8       __acrt_initialize          0000000180003fe8 f   MSVCRT:ucrt_stubs.obj
 0001:00002fe8       __acrt_thread_attach       0000000180003fe8 f   MSVCRT:ucrt_stubs.obj
 0001:00002fe8       __acrt_thread_detach       0000000180003fe8 f   MSVCRT:ucrt_stubs.obj
 0001:00002fe8       __acrt_uninitialize        0000000180003fe8 f   MSVCRT:ucrt_stubs.obj
 0001:00002fe8       __acrt_uninitialize_critical 0000000180003fe8 f   MSVCRT:ucrt_stubs.obj
 0001:00002fe8       __scrt_stub_for_acrt_initialize 0000000180003fe8 f   MSVCRT:ucrt_stubs.obj
 0001:00002fe8       __scrt_stub_for_acrt_thread_attach 0000000180003fe8 f   MSVCRT:ucrt_stubs.obj
 0001:00002fe8       __scrt_stub_for_acrt_thread_detach 0000000180003fe8 f   MSVCRT:ucrt_stubs.obj
 0001:00002fe8       __scrt_stub_for_acrt_uninitialize 0000000180003fe8 f   MSVCRT:ucrt_stubs.obj
 0001:00002fe8       __scrt_stub_for_acrt_uninitialize_critical 0000000180003fe8 f   MSVCRT:ucrt_stubs.obj
 0001:00002fe8       __vcrt_initialize          0000000180003fe8 f   MSVCRT:ucrt_stubs.obj
 0001:00002fe8       __vcrt_thread_attach       0000000180003fe8 f   MSVCRT:ucrt_stubs.obj
 0001:00002fe8       __vcrt_thread_detach       0000000180003fe8 f   MSVCRT:ucrt_stubs.obj
 0001:00002fe8       __vcrt_uninitialize        0000000180003fe8 f   MSVCRT:ucrt_stubs.obj
 0001:00002fe8       __vcrt_uninitialize_critical 0000000180003fe8 f   MSVCRT:ucrt_stubs.obj
 0001:00002fec       __scrt_stub_for_is_c_termination_complete 0000000180003fec f   MSVCRT:ucrt_stubs.obj
 0001:00002fec       _is_c_termination_complete 0000000180003fec f   MSVCRT:ucrt_stubs.obj
 0001:00003000       _guard_dispatch_icall_nop  0000000180004000 f   MSVCRT:guard_dispatch.obj
 0001:00003020       _guard_xfg_dispatch_icall_nop 0000000180004020 f   MSVCRT:guard_xfg_dispatch.obj
 0002:00000000       __imp_RtlCaptureContext    0000000180005000     kernel32:KERNEL32.dll
 0002:00000008       __imp_RtlLookupFunctionEntry 0000000180005008     kernel32:KERNEL32.dll
 0002:00000010       __imp_RtlVirtualUnwind     0000000180005010     kernel32:KERNEL32.dll
 0002:00000018       __imp_UnhandledExceptionFilter 0000000180005018     kernel32:KERNEL32.dll
 0002:00000020       __imp_SetUnhandledExceptionFilter 0000000180005020     kernel32:KERNEL32.dll
 0002:00000028       __imp_GetCurrentProcess    0000000180005028     kernel32:KERNEL32.dll
 0002:00000030       __imp_TerminateProcess     0000000180005030     kernel32:KERNEL32.dll
 0002:00000038       __imp_IsProcessorFeaturePresent 0000000180005038     kernel32:KERNEL32.dll
 0002:00000040       __imp_CloseHandle          0000000180005040     kernel32:KERNEL32.dll
 0002:00000048       __imp_InitializeCriticalSectionAndSpinCount 0000000180005048     kernel32:KERNEL32.dll
 0002:00000050       __imp_DeleteCriticalSection 0000000180005050     kernel32:KERNEL32.dll
 0002:00000058       __imp_CreateEventW         0000000180005058     kernel32:KERNEL32.dll
 0002:00000060       __imp_GetModuleHandleW     0000000180005060     kernel32:KERNEL32.dll
 0002:00000068       __imp_GetProcAddress       0000000180005068     kernel32:KERNEL32.dll
 0002:00000070       __imp_IsDebuggerPresent    0000000180005070     kernel32:KERNEL32.dll
 0002:00000078       __imp_QueryPerformanceCounter 0000000180005078     kernel32:KERNEL32.dll
 0002:00000080       __imp_GetCurrentProcessId  0000000180005080     kernel32:KERNEL32.dll
 0002:00000088       __imp_GetCurrentThreadId   0000000180005088     kernel32:KERNEL32.dll
 0002:00000090       __imp_GetSystemTimeAsFileTime 0000000180005090     kernel32:KERNEL32.dll
 0002:00000098       __imp_DisableThreadLibraryCalls 0000000180005098     kernel32:KERNEL32.dll
 0002:000000a0       __imp_InitializeSListHead  00000001800050a0     kernel32:KERNEL32.dll
 0002:000000a8       \177KERNEL32_NULL_THUNK_DATA 00000001800050a8     kernel32:KERNEL32.dll
 0002:000000b0       __imp_memcpy               00000001800050b0     vcruntime:VCRUNTIME140.dll
 0002:000000b8       __imp_memset               00000001800050b8     vcruntime:VCRUNTIME140.dll
 0002:000000c0       __imp_strchr               00000001800050c0     vcruntime:VCRUNTIME140.dll
 0002:000000c8       __imp___C_specific_handler 00000001800050c8     vcruntime:VCRUNTIME140.dll
 0002:000000d0       __imp___std_type_info_destroy_list 00000001800050d0     vcruntime:VCRUNTIME140.dll
 0002:000000d8       \177VCRUNTIME140_NULL_THUNK_DATA 00000001800050d8     vcruntime:VCRUNTIME140.dll
 0002:000000e0       __imp__errno               00000001800050e0     ucrt:api-ms-win-crt-runtime-l1-1-0.dll
 0002:000000e8       __imp_exit                 00000001800050e8     ucrt:api-ms-win-crt-runtime-l1-1-0.dll
 0002:000000f0       __imp__cexit               00000001800050f0     ucrt:api-ms-win-crt-runtime-l1-1-0.dll
 0002:000000f8       __imp__crt_atexit          00000001800050f8     ucrt:api-ms-win-crt-runtime-l1-1-0.dll
 0002:00000100       __imp__execute_onexit_table 0000000180005100     ucrt:api-ms-win-crt-runtime-l1-1-0.dll
 0002:00000108       __imp__register_onexit_function 0000000180005108     ucrt:api-ms-win-crt-runtime-l1-1-0.dll
 0002:00000110       __imp__initialize_onexit_table 0000000180005110     ucrt:api-ms-win-crt-runtime-l1-1-0.dll
 0002:00000118       __imp__initialize_narrow_environment 0000000180005118     ucrt:api-ms-win-crt-runtime-l1-1-0.dll
 0002:00000120       __imp__configure_narrow_argv 0000000180005120     ucrt:api-ms-win-crt-runtime-l1-1-0.dll
 0002:00000128       __imp__seh_filter_dll      0000000180005128     ucrt:api-ms-win-crt-runtime-l1-1-0.dll
 0002:00000130       __imp__initterm_e          0000000180005130     ucrt:api-ms-win-crt-runtime-l1-1-0.dll
 0002:00000138       __imp__initterm            0000000180005138     ucrt:api-ms-win-crt-runtime-l1-1-0.dll
 0002:00000140       \177api-ms-win-crt-runtime-l1-1-0_NULL_THUNK_DATA 0000000180005140     ucrt:api-ms-win-crt-runtime-l1-1-0.dll
 0002:00000148       __imp___acrt_iob_func      0000000180005148     ucrt:api-ms-win-crt-stdio-l1-1-0.dll
 0002:00000150       __imp_fflush               0000000180005150     ucrt:api-ms-win-crt-stdio-l1-1-0.dll
 0002:00000158       __imp___stdio_common_vsprintf 0000000180005158     ucrt:api-ms-win-crt-stdio-l1-1-0.dll
 0002:00000160       __imp___stdio_common_vfprintf 0000000180005160     ucrt:api-ms-win-crt-stdio-l1-1-0.dll
 0002:00000168       \177api-ms-win-crt-stdio-l1-1-0_NULL_THUNK_DATA 0000000180005168     ucrt:api-ms-win-crt-stdio-l1-1-0.dll
 0002:00000170       __imp_strcmp               0000000180005170     ucrt:api-ms-win-crt-string-l1-1-0.dll
 0002:00000178       __imp__strdup              0000000180005178     ucrt:api-ms-win-crt-string-l1-1-0.dll
 0002:00000178       __imp_strdup               0000000180005178     ucrt:api-ms-win-crt-string-l1-1-0.dll
 0002:00000180       __imp_strlen               0000000180005180     ucrt:api-ms-win-crt-string-l1-1-0.dll
 0002:00000188       __imp_strncpy              0000000180005188     ucrt:api-ms-win-crt-string-l1-1-0.dll
 0002:00000190       \177api-ms-win-crt-string-l1-1-0_NULL_THUNK_DATA 0000000180005190     ucrt:api-ms-win-crt-string-l1-1-0.dll
 0002:00000198       __guard_check_icall_fptr   0000000180005198     MSVCRT:guard_support.obj
 0002:000001a0       __guard_xfg_check_icall_fptr 00000001800051a0     MSVCRT:guard_support.obj
 0002:000001a8       __guard_dispatch_icall_fptr 00000001800051a8     MSVCRT:guard_support.obj
 0002:000001b0       __guard_xfg_dispatch_icall_fptr 00000001800051b0     MSVCRT:guard_support.obj
 0002:000001b8       __guard_xfg_table_dispatch_icall_fptr 00000001800051b8     MSVCRT:guard_support.obj
 0002:000001c0       __castguard_check_failure_os_handled_fptr 00000001800051c0     MSVCRT:guard_support.obj
 0002:000001c8       __guard_memcpy_fptr        00000001800051c8     vcruntime:softmemtag.obj
 0002:000001d0       __xc_a                     00000001800051d0     MSVCRT:initializers.obj
 0002:000001d8       __xc_z                     00000001800051d8     MSVCRT:initializers.obj
 0002:000001e0       __xi_a                     00000001800051e0     MSVCRT:initializers.obj
 0002:000001f0       __xi_z                     00000001800051f0     MSVCRT:initializers.obj
 0002:000001f8       __xl_a                     00000001800051f8     MSVCRT:tlssup.obj
 0002:00000200       __xl_z                     0000000180005200     MSVCRT:tlssup.obj
 0002:00000208       __xp_a                     0000000180005208     MSVCRT:initializers.obj
 0002:00000210       __xp_z                     0000000180005210     MSVCRT:initializers.obj
 0002:00000218       __xt_a                     0000000180005218     MSVCRT:initializers.obj
 0002:00000220       __xt_z                     0000000180005220     MSVCRT:initializers.obj
 0002:00000230       g_refKindStr               0000000180005230     libpopframe008.obj
 0002:000003e0       ??_C@_09BPLDFGCI@unknown_0@ 00000001800053e0     libpopframe008.obj
 0002:000003f0       ??_C@_0BL@FPNMECJD@JVMTI_HEAP_REFERENCE_CLASS@ 00000001800053f0     libpopframe008.obj
 0002:00000410       ??_C@_0BL@FKGKKLNM@JVMTI_HEAP_REFERENCE_FIELD@ 0000000180005410     libpopframe008.obj
 0002:00000430       ??_C@_0CD@CAEHCFJF@JVMTI_HEAP_REFERENCE_ARRAY_ELEM@ 0000000180005430     libpopframe008.obj
 0002:00000458       ??_C@_0CC@DNEBMCNK@JVMTI_HEAP_REFERENCE_CLASS_LOAD@ 0000000180005458     libpopframe008.obj
 0002:00000480       ??_C@_0BN@CJMIPEBB@JVMTI_HEAP_REFERENCE_SIGNERS@ 0000000180005480     libpopframe008.obj
 0002:000004a0       ??_C@_0CH@HBOIDPEB@JVMTI_HEAP_REFERENCE_PROTECTION@ 00000001800054a0     libpopframe008.obj
 0002:000004c8       ??_C@_0BP@MDKGDGKL@JVMTI_HEAP_REFERENCE_INTERFACE@ 00000001800054c8     libpopframe008.obj
 0002:000004e8       ??_C@_0CC@JJMIHNJH@JVMTI_HEAP_REFERENCE_STATIC_FIE@ 00000001800054e8     libpopframe008.obj
 0002:00000510       ??_C@_0CD@IDHEEGID@JVMTI_HEAP_REFERENCE_CONSTANT_P@ 0000000180005510     libpopframe008.obj
 0002:00000538       ??_C@_0CA@EFFCHNG@JVMTI_HEAP_REFERENCE_SUPERCLASS@ 0000000180005538     libpopframe008.obj
 0002:00000558       ??_C@_0L@PCDFHGCJ@unknown_11@ 0000000180005558     libpopframe008.obj
 0002:00000568       ??_C@_0L@NJBICFOK@unknown_12@ 0000000180005568     libpopframe008.obj
 0002:00000578       ??_C@_0L@MAADBEKL@unknown_13@ 0000000180005578     libpopframe008.obj
 0002:00000588       ??_C@_0L@IPECICGM@unknown_14@ 0000000180005588     libpopframe008.obj
 0002:00000598       ??_C@_0L@JGFJLDCN@unknown_15@ 0000000180005598     libpopframe008.obj
 0002:000005a8       ??_C@_0L@LNHEOAOO@unknown_16@ 00000001800055a8     libpopframe008.obj
 0002:000005b8       ??_C@_0L@KEGPNBKP@unknown_17@ 00000001800055b8     libpopframe008.obj
 0002:000005c8       ??_C@_0L@CDPHMNGA@unknown_18@ 00000001800055c8     libpopframe008.obj
 0002:000005d8       ??_C@_0L@DKOMPMCB@unknown_19@ 00000001800055d8     libpopframe008.obj
 0002:000005e8       ??_C@_0L@OJGIPJDB@unknown_20@ 00000001800055e8     libpopframe008.obj
 0002:000005f8       ??_C@_0CA@KAOFNDEM@JVMTI_HEAP_REFERENCE_JNI_GLOBAL@ 00000001800055f8     libpopframe008.obj
 0002:00000618       ??_C@_0CC@HPFAJBK@JVMTI_HEAP_REFERENCE_SYSTEM_CLA@ 0000000180005618     libpopframe008.obj
 0002:00000640       ??_C@_0BN@FDEGFOHC@JVMTI_HEAP_REFERENCE_MONITOR@ 0000000180005640     libpopframe008.obj
 0002:00000660       ??_C@_0CB@HKIBCMAJ@JVMTI_HEAP_REFERENCE_STACK_LOCA@ 0000000180005660     libpopframe008.obj
 0002:00000688       ??_C@_0BP@EAACMMOE@JVMTI_HEAP_REFERENCE_JNI_LOCAL@ 0000000180005688     libpopframe008.obj
 0002:000006a8       ??_C@_0BM@IJDEOGOE@JVMTI_HEAP_REFERENCE_THREAD@ 00000001800056a8     libpopframe008.obj
 0002:000006c8       ??_C@_0BL@EDGPPKC@JVMTI_HEAP_REFERENCE_OTHER@ 00000001800056c8     libpopframe008.obj
 0002:000006e4       ??_C@_04BCJPDBDA@Code@     00000001800056e4     libpopframe008.obj
 0002:000006f0       ??_C@_0BA@OCLMCFKC@LineNumberTable@ 00000001800056f0     libpopframe008.obj
 0002:00000700       ??_C@_0BD@CPAEPILC@LocalVariableTable@ 0000000180005700     libpopframe008.obj
 0002:00000718       ??_C@_0BH@NMBDNHBD@LocalVariableTypeTable@ 0000000180005718     libpopframe008.obj
 0002:00000730       ??_C@_0O@HIHEEDNJ@StackMapTable@ 0000000180005730     libpopframe008.obj
 0002:00000740       ??_C@_03GAEACAIP@?$CI?$CJV@ 0000000180005740     libpopframe008.obj
 0002:00000748       ??_C@_0CM@HDCCPGMD@Lnsk?1jvmti?1PopFrame?1popframe008@ 0000000180005748     libpopframe008.obj
 0002:00000774       ??_C@_01GFHCPBMG@C@        0000000180005774     libpopframe008.obj
 0002:00000778       ??_C@_01HMGJMAIH@B@        0000000180005778     libpopframe008.obj
 0002:0000077c       ??_C@_01FHEEJDEE@A@        000000018000577c     libpopframe008.obj
 0002:00000780       ??_C@_03LGMJKEGG@run@      0000000180005780     libpopframe008.obj
 0002:00000788       ??_C@_0L@HCDIAMJG@?9?5?$CFs?0?5?$CFd?3?5@ 0000000180005788     libpopframe008.obj
 0002:000007a0       ??_C@_0JI@HLPECLFI@?$CD?5?4?4?4?6?$CD?5ERROR?3?5too?5many?5complai@ 00000001800057a0     libpopframe008.obj
 0002:00000840       ??_C@_0ED@JNEKCCOB@The?5following?5fake?5exception?5st@ 0000000180005840     libpopframe008.obj
 0002:00000888       ??_C@_0CN@FCNMDFBH@nsk?4share?4Fake_Exception_for_RU@ 0000000180005888     libpopframe008.obj
 0002:000008b8       ??_C@_08PGFFNAEI@?$CI?$CFs?3?$CFd?$CJ?5@ 00000001800058b8     libpopframe008.obj
 0002:000008c8       ??_C@_0DP@IENMAEGI@s?2test?2hotspot?2jtreg?2vmTestbase@ 00000001800058c8     libpopframe008.obj
 0002:00000908       ??_C@_0BL@NDJLFFJB@?7at?5nsk_lvcomplain?$CI?$CFs?3?$CFd?$CJ?6@ 0000000180005908     libpopframe008.obj
 0002:00000928       ??_C@_0BC@JOOKAFKF@?$CD?5ERROR?3?5?$CFs?0?5?$CFd?3?5@ 0000000180005928     libpopframe008.obj
 0002:00000940       ??_C@_09KJEAHMEH@?$CD?5ERROR?3?5@ 0000000180005940     libpopframe008.obj
 0002:0000094c       ??_C@_02GPIOPFAK@?$DO?$DO@ 000000018000594c     libpopframe008.obj
 0002:00000950       ??_C@_02FODMEDOG@?$DM?$DM@ 0000000180005950     libpopframe008.obj
 0002:00000954       ??_C@_02DJGKEECL@?4?4@     0000000180005954     libpopframe008.obj
 0002:00000958       ??_C@_0O@CJPGJOAF@?9?5?$CFs?0?5?$CFd?3?5?$CFs?5@ 0000000180005958     libpopframe008.obj
 0002:00000968       ??_C@_0CB@IAKPDOIC@?$CD?5?5?5verified?5assertion?5is?5FALSE@ 0000000180005968     libpopframe008.obj
 0002:00000990       ??_C@_0CO@LGONDEPD@stdout?3?5fflush?5failed?5?9?5err?$DN?$CFd?5@ 0000000180005990     libpopframe008.obj
 0002:000009c0       ??_C@_0CO@KBGKJPBD@stderr?3?5fflush?5failed?5?9?5err?$DN?$CFd?5@ 00000001800059c0     libpopframe008.obj
 0002:000009f0       ??_C@_0BB@JCNMKLLK@JVMTI_ERROR_NONE@ 00000001800059f0     libpopframe008.obj
 0002:00000a08       ??_C@_0BL@LDIMKLPH@JVMTI_ERROR_INVALID_THREAD@ 0000000180005a08     libpopframe008.obj
 0002:00000a28       ??_C@_0CB@PJFPAIKJ@JVMTI_ERROR_INVALID_THREAD_GROU@ 0000000180005a28     libpopframe008.obj
 0002:00000a50       ??_C@_0BN@LLMKHMNF@JVMTI_ERROR_INVALID_PRIORITY@ 0000000180005a50     libpopframe008.obj
 0002:00000a70       ??_C@_0CB@MBOFKAGB@JVMTI_ERROR_THREAD_NOT_SUSPENDE@ 0000000180005a70     libpopframe008.obj
 0002:00000a98       ??_C@_0BN@FABOLPBI@JVMTI_ERROR_THREAD_SUSPENDED@ 0000000180005a98     libpopframe008.obj
 0002:00000ab8       ??_C@_0BN@FDGNOBJM@JVMTI_ERROR_THREAD_NOT_ALIVE@ 0000000180005ab8     libpopframe008.obj
 0002:00000ad8       ??_C@_0BL@GOBIFKNJ@JVMTI_ERROR_INVALID_OBJECT@ 0000000180005ad8     libpopframe008.obj
 0002:00000af8       ??_C@_0BK@FCMAJPPC@JVMTI_ERROR_INVALID_CLASS@ 0000000180005af8     libpopframe008.obj
 0002:00000b18       ??_C@_0BP@IKLLBKEB@JVMTI_ERROR_CLASS_NOT_PREPARED@ 0000000180005b18     libpopframe008.obj
 0002:00000b38       ??_C@_0BN@KLPPLKG@JVMTI_ERROR_INVALID_METHODID@ 0000000180005b38     libpopframe008.obj
 0002:00000b58       ??_C@_0BN@BCEKOKND@JVMTI_ERROR_INVALID_LOCATION@ 0000000180005b58     libpopframe008.obj
 0002:00000b78       ??_C@_0BM@DFDGPME@JVMTI_ERROR_INVALID_FIELDID@ 0000000180005b78     libpopframe008.obj
 0002:00000b98       ??_C@_0BL@NELIEPEC@JVMTI_ERROR_NO_MORE_FRAMES@ 0000000180005b98     libpopframe008.obj
 0002:00000bb8       ??_C@_0BJ@BDBECFDM@JVMTI_ERROR_OPAQUE_FRAME@ 0000000180005bb8     libpopframe008.obj
 0002:00000bd8       ??_C@_0BK@MIIFNLOB@JVMTI_ERROR_TYPE_MISMATCH@ 0000000180005bd8     libpopframe008.obj
 0002:00000bf8       ??_C@_0BJ@HPCAOILC@JVMTI_ERROR_INVALID_SLOT@ 0000000180005bf8     libpopframe008.obj
 0002:00000c18       ??_C@_0BG@CHILOPNI@JVMTI_ERROR_DUPLICATE@ 0000000180005c18     libpopframe008.obj
 0002:00000c30       ??_C@_0BG@DIEMLHKM@JVMTI_ERROR_NOT_FOUND@ 0000000180005c30     libpopframe008.obj
 0002:00000c48       ??_C@_0BM@NHMCKHOB@JVMTI_ERROR_INVALID_MONITOR@ 0000000180005c48     libpopframe008.obj
 0002:00000c68       ??_C@_0BO@PPEDAJGL@JVMTI_ERROR_NOT_MONITOR_OWNER@ 0000000180005c68     libpopframe008.obj
 0002:00000c88       ??_C@_0BG@FCAIPEID@JVMTI_ERROR_INTERRUPT@ 0000000180005c88     libpopframe008.obj
 0002:00000ca0       ??_C@_0CB@EGDBNKOI@JVMTI_ERROR_INVALID_CLASS_FORMA@ 0000000180005ca0     libpopframe008.obj
 0002:00000cc8       ??_C@_0CG@DGKOGIAL@JVMTI_ERROR_CIRCULAR_CLASS_DEFI@ 0000000180005cc8     libpopframe008.obj
 0002:00000cf0       ??_C@_0BP@ICEALPKC@JVMTI_ERROR_FAILS_VERIFICATION@ 0000000180005cf0     libpopframe008.obj
 0002:00000d10       ??_C@_0DC@JDACLMIO@JVMTI_ERROR_UNSUPPORTED_REDEFIN@ 0000000180005d10     libpopframe008.obj
 0002:00000d48       ??_C@_0DE@GKDKNOMJ@JVMTI_ERROR_UNSUPPORTED_REDEFIN@ 0000000180005d48     libpopframe008.obj
 0002:00000d80       ??_C@_0BO@LAFKIOG@JVMTI_ERROR_INVALID_TYPESTATE@ 0000000180005d80     libpopframe008.obj
 0002:00000da0       ??_C@_0DH@INDGCLLB@JVMTI_ERROR_UNSUPPORTED_REDEFIN@ 0000000180005da0     libpopframe008.obj
 0002:00000dd8       ??_C@_0DE@NHEOMMGI@JVMTI_ERROR_UNSUPPORTED_REDEFIN@ 0000000180005dd8     libpopframe008.obj
 0002:00000e10       ??_C@_0CA@EKPNJOEP@JVMTI_ERROR_UNSUPPORTED_VERSION@ 0000000180005e10     libpopframe008.obj
 0002:00000e30       ??_C@_0BN@OFFMAHHL@JVMTI_ERROR_NAMES_DONT_MATCH@ 0000000180005e30     libpopframe008.obj
 0002:00000e50       ??_C@_0DN@HHBBLAKE@JVMTI_ERROR_UNSUPPORTED_REDEFIN@ 0000000180005e50     libpopframe008.obj
 0002:00000e90       ??_C@_0DO@HMBGBGNA@JVMTI_ERROR_UNSUPPORTED_REDEFIN@ 0000000180005e90     libpopframe008.obj
 0002:00000ed0       ??_C@_0BP@PBECGKHJ@JVMTI_ERROR_UNMODIFIABLE_CLASS@ 0000000180005ed0     libpopframe008.obj
 0002:00000ef0       ??_C@_0BK@CANILEHF@JVMTI_ERROR_NOT_AVAILABLE@ 0000000180005ef0     libpopframe008.obj
 0002:00000f10       ??_C@_0CE@INJKMEFK@JVMTI_ERROR_MUST_POSSESS_CAPABI@ 0000000180005f10     libpopframe008.obj
 0002:00000f38       ??_C@_0BJ@LBFPFPDM@JVMTI_ERROR_NULL_POINTER@ 0000000180005f38     libpopframe008.obj
 0002:00000f58       ??_C@_0BP@CHJPNNEM@JVMTI_ERROR_ABSENT_INFORMATION@ 0000000180005f58     libpopframe008.obj
 0002:00000f78       ??_C@_0BP@OMFMNLC@JVMTI_ERROR_INVALID_EVENT_TYPE@ 0000000180005f78     libpopframe008.obj
 0002:00000f98       ??_C@_0BN@BIBNPHHO@JVMTI_ERROR_ILLEGAL_ARGUMENT@ 0000000180005f98     libpopframe008.obj
 0002:00000fb8       ??_C@_0BK@KKNDHDCE@JVMTI_ERROR_NATIVE_METHOD@ 0000000180005fb8     libpopframe008.obj
 0002:00000fd8       ??_C@_0BK@PMKCFHAE@JVMTI_ERROR_OUT_OF_MEMORY@ 0000000180005fd8     libpopframe008.obj
 0002:00000ff8       ??_C@_0BK@NNJBDMNB@JVMTI_ERROR_ACCESS_DENIED@ 0000000180005ff8     libpopframe008.obj
 0002:00001018       ??_C@_0BI@GHECLMNC@JVMTI_ERROR_WRONG_PHASE@ 0000000180006018     libpopframe008.obj
 0002:00001030       ??_C@_0BF@OLIHJOII@JVMTI_ERROR_INTERNAL@ 0000000180006030     libpopframe008.obj
 0002:00001048       ??_C@_0BO@EOHGKJHI@JVMTI_ERROR_UNATTACHED_THREAD@ 0000000180006048     libpopframe008.obj
 0002:00001068       ??_C@_0CA@LKHFDACL@JVMTI_ERROR_INVALID_ENVIRONMENT@ 0000000180006068     libpopframe008.obj
 0002:00001088       ??_C@_0BA@MMFHLOKK@?$DMunknown?5error?$DO@ 0000000180006088     libpopframe008.obj
 0002:00001098       ??_C@_0CF@CBHOKDB@throwable?5?$DN?5jni?9?$DOExceptionOccur@ 0000000180006098     libpopframe008.obj
 0002:000010c0       ??_C@_03OFAPEBGM@?$CFs?6@  00000001800060c0     libpopframe008.obj
 0002:000010c8       ??_C@_0DM@LPIGEGNJ@s?2test?2hotspot?2jtreg?2vmTestbase@ 00000001800060c8     libpopframe008.obj
 0002:00001108       ??_C@_0CC@NFCNPEPK@Exception?5in?5JNI?5call?5?$CIcleared?$CJ@ 0000000180006108     libpopframe008.obj
 0002:00001130       ??_C@_0BJ@IBAKFIKF@jni?9?$DOExceptionDescribe?$CI?$CJ@ 0000000180006130     libpopframe008.obj
 0002:00001150       ??_C@_0BG@GGKALKMH@jni?9?$DOExceptionClear?$CI?$CJ@ 0000000180006150     libpopframe008.obj
 0002:00001168       ??_C@_0CF@JMGFGJLJ@?$CD?5?5?5verified?5JNI?5assertion?5is?5F@ 0000000180006168     libpopframe008.obj
 0002:00001190       ??_C@_0CB@MLNJNCLJ@?5?5jvmti?5error?3?5code?$DN?$CFd?0?5name?$DN?$CFs@ 0000000180006190     libpopframe008.obj
 0002:000011b8       ??_C@_0CD@OHBGDKMK@?$CD?5?5?5jvmti?5error?3?5code?$DN?$CFd?0?5name?$DN@ 00000001800061b8     libpopframe008.obj
 0002:000011e0       ??_C@_0CG@JNNCGPHB@?$CD?5?5?5error?5expected?3?5code?$DN?$CFd?0?5na@ 00000001800061e0     libpopframe008.obj
 0002:00001210       ??_C@_0EB@IMGKPCGE@?$CIstr_obj?5?$DN?5jni?9?$DONewStringUTF?$CIco@ 0000000180006210     libpopframe008.obj
 0002:00001260       ??_C@_0EA@HFOGGBCC@s?2test?2hotspot?2jtreg?2vmTestbase@ 0000000180006260     libpopframe008.obj
 0002:000012a0       ??_C@_05KKCIMGE@error@     00000001800062a0     libpopframe008.obj
 0002:000012b0       ??_C@_0EA@PNBCDMOA@s?2test?2hotspot?2jtreg?2vmTestbase@ 00000001800062b0     libpopframe008.obj
 0002:000012f0       ??_C@_0DI@ILAHDLMP@?$CI?$CKagentThreadProc?$CJ?$CIjvmti_env?0?5a@ 00000001800062f0     libpopframe008.obj
 0002:00001328       ??_C@_0BD@KDBALNLB@JVMTI?5agent?5thread@ 0000000180006328     libpopframe008.obj
 0002:00001340       ??_C@_0BB@NOKBFPFO@java?1lang?1Thread@ 0000000180006340     libpopframe008.obj
 0002:00001354       ??_C@_06FALKBLGB@?$DMinit?$DO@ 0000000180006354     libpopframe008.obj
 0002:00001360       ??_C@_0BG@IKDDPPGD@?$CILjava?1lang?1String?$DL?$CJV@ 0000000180006360     libpopframe008.obj
 0002:00001380       ??_C@_0EB@IFJBFEKC@?$CIthreadClass?5?$DN?5jni_env?9?$DOFindCla@ 0000000180006380     libpopframe008.obj
 0002:000013d0       ??_C@_0GF@FGFIBKKL@?$CIthreadCtor?5?$DN?5jni_env?9?$DOGetMetho@ 00000001800063d0     libpopframe008.obj
 0002:00001438       ??_C@_0DN@NCPDJLOG@?$CIthreadName?5?$DN?5jni_env?9?$DONewStrin@ 0000000180006438     libpopframe008.obj
 0002:00001480       ??_C@_0FE@PFKODBGC@?$CIthreadObject?5?$DN?5jni_env?9?$DONewObj@ 0000000180006480     libpopframe008.obj
 0002:000014e0       ??_C@_0ED@HOBAHHJI@?$CIthreadGlobalRef?5?$DN?5jni_env?9?$DONew@ 00000001800064e0     libpopframe008.obj
 0002:00001530       ??_C@_0FN@HNJJAHFC@jvmti_env?9?$DORunAgentThread?$CIagent@ 0000000180006530     libpopframe008.obj
 0002:00001590       ??_C@_0EA@MOJDNKDF@Debuggee?5status?5sync?5aborted?5be@ 0000000180006590     libpopframe008.obj
 0002:000015d0       ??_C@_0EA@EEOEJAEN@status?5?$DN?5syncDebuggeeStatus?$CIjni@ 00000001800065d0     libpopframe008.obj
 0002:00001610       ??_C@_0BL@JBCFNBMB@nsk_jvmti_resetAgentData?$CI?$CJ@ 0000000180006610     libpopframe008.obj
 0002:00001630       ??_C@_0EL@LPBEELIP@s?2test?2hotspot?2jtreg?2vmTestbase@ 0000000180006630     libpopframe008.obj
 0002:00001680       ??_C@_0CK@JDAMFDMJ@jvmti?9?$DOSetTag?$CIo?0?5tag?$CJ?5?$DN?$DN?5JVMTI_@ 0000000180006680     libpopframe008.obj
 0002:000016b0       ??_C@_0CC@DAMNHKNI@Can?8t?5set?5tag?5?$CFli?5for?5object?5?$CFl@ 00000001800066b0     libpopframe008.obj
 0002:000016d8       ??_C@_0DL@HAJPNKEF@jvmti?9?$DOGetObjectHashCode?$CIo?0?5?$CGha@ 00000001800066d8     libpopframe008.obj
 0002:00001718       ??_C@_0BL@JFPIEOBF@Can?8t?5get?5hash?5object?5?$CFlx?6@ 0000000180006718     libpopframe008.obj
 0002:00001738       ??_C@_0BG@DICPHBKN@setTag?3?5?$CF08x?5?$DM?9?5?$CF?53li@ 0000000180006738     libpopframe008.obj
 0002:00001750       ??_C@_0DH@FCEEBDMJ@?$CIs?5?$DN?5jni?9?$DOGetStringUTFChars?$CIsIn@ 0000000180006750     libpopframe008.obj
 0002:00001788       ??_C@_0BJ@OKKGHDCN@Can?8t?5get?5string?5at?5?$CF?$CDp?6@ 0000000180006788     libpopframe008.obj
 0002:000017a8       ??_C@_0BP@EKFLGGFJ@Can?8t?5get?5string?5at?5?$CF?$CDp?3?5null?6@ 00000001800067a8     libpopframe008.obj
 0002:000017c8       ??_C@_06ICODBHCL@?5?1?1?5?$CFs@ 00000001800067c8     libpopframe008.obj
 0002:000017d0       ??_C@_0DB@KGFPLEGO@?$CIr?5?$DN?5jvmti?9?$DOGetTag?$CIo?0?5?$CGtag?$CJ?$CJ?5?$DN?$DN@ 00000001800067d0     libpopframe008.obj
 0002:00001808       ??_C@_0CO@PDAGBCGJ@Can?8t?5GetTag?5for?5object?5?$CFlx?4?5Re@ 0000000180006808     libpopframe008.obj
 0002:00001838       ??_C@_0CH@HPEODOHC@TEST_BUG?3?5Max?4?5number?5of?5refs?5r@ 0000000180006838     libpopframe008.obj
 0002:00001860       ??_C@_0DI@PHFCABIM@?$CIr?5?$DN?5jvmti?9?$DOGetTag?$CIfrom?0?5?$CGtagFr@ 0000000180006860     libpopframe008.obj
 0002:00001898       ??_C@_0DI@MDEGFNKD@TEST_BUG?3?5Can?8t?5GetTag?5for?5obje@ 0000000180006898     libpopframe008.obj
 0002:000018d0       ??_C@_0DE@MLELJAHM@?$CIr?5?$DN?5jvmti?9?$DOGetTag?$CIto?0?5?$CGtagTo?$CJ?$CJ@ 00000001800068d0     libpopframe008.obj
 0002:00001908       ??_C@_0DI@HDMIALG@?$CIGetMethodDeclaringClass?$CD?$CFd?$CJ?5un@ 0000000180006908     libpopframe008.obj
 0002:00001940       ??_C@_0DC@CKFFJKGO@?$CIGetClassSignature?$CD?$CFd?$CJ?5unexpect@ 0000000180006940     libpopframe008.obj
 0002:00001978       ??_C@_0CO@BDGJACHG@?$CIGetMethodName?$CD?$CFd?$CJ?5unexpected?5e@ 0000000180006978     libpopframe008.obj
 0002:000019a8       ??_C@_0BN@MDDAMKHB@?$CI?$CFd?$CJ?5wrong?5class?5sig?3?5?$CC?$CFs?$CC?0?6@ 00000001800069a8     libpopframe008.obj
 0002:000019c8       ??_C@_0BB@GMOCCHAJ@?5expected?3?5?$CC?$CFs?$CC?6@ 00000001800069c8     libpopframe008.obj
 0002:000019e0       ??_C@_0BO@LOALJDPL@?$CI?$CFd?$CJ?5wrong?5method?5name?3?5?$CC?$CFs?$CC?0@ 00000001800069e0     libpopframe008.obj
 0002:00001a00       ??_C@_0BN@HMBLKCLB@?$CI?$CFd?$CJ?5wrong?5method?5sig?3?5?$CC?$CFs?$CC?0@ 0000000180006a00     libpopframe008.obj
 0002:00001a20       ??_C@_0BP@IJBNPKOG@?$CI?$CFd?$CJ?5wrong?5location?3?50x?$CFx?$CF08x?0@ 0000000180006a20     libpopframe008.obj
 0002:00001a40       ??_C@_0BB@GNDCHEPL@?5expected?3?50x?$CFx?6@ 0000000180006a40     libpopframe008.obj
 0002:00001a58       ??_C@_0O@HJHLBNFC@?$DO?$DO?$DO?5?$CC?$CFs?4?$CFs?$CFs?$CC@ 0000000180006a58     libpopframe008.obj
 0002:00001a68       ??_C@_0BG@MHMCCJEK@?0?5location?3?50x?$CFx?$CF08x?6@ 0000000180006a68     libpopframe008.obj
 0002:00001a80       ??_C@_0CI@ODAHCOFC@bp?3?5don?8t?5know?5where?5we?5get?5cal@ 0000000180006a80     libpopframe008.obj
 0002:00001aa8       ??_C@_0BF@EFEMDGBO@?$DO?$DO?$DO?5breakpoint?5in?5D?6@ 0000000180006aa8     libpopframe008.obj
 0002:00001ac0       ??_C@_0CN@MNGFMGHL@?$CIClearBreakpoint?$CJ?5unexpected?5er@ 0000000180006ac0     libpopframe008.obj
 0002:00001af0       ??_C@_0CE@FMDJGKKD@Cannot?5enable?5single?5step?3?5?$CFs?5?$CI@ 0000000180006af0     libpopframe008.obj
 0002:00001b18       ??_C@_0CG@LNOCPLAB@?$CIPopFrame?$CJ?5unexpected?5error?3?5?$CFs@ 0000000180006b18     libpopframe008.obj
 0002:00001b40       ??_C@_0CJ@GDAKNPPK@?$DO?$DO?$DO?5poped?5?$CFd?5frames?5till?5method@ 0000000180006b40     libpopframe008.obj
 0002:00001b70       ??_C@_0CF@OAOLHEMH@Cannot?5disable?5single?5step?3?5?$CFs?5@ 0000000180006b70     libpopframe008.obj
 0002:00001b98       ??_C@_09OPJEJKBL@printdump@ 0000000180006b98     libpopframe008.obj
 0002:00001ba8       ??_C@_0CJ@KCDEKOCJ@Wrong?5result?5of?5a?5valid?5call?5to@ 0000000180006ba8     libpopframe008.obj
 0002:00001bd8       ??_C@_0DG@LAJPGIIE@?$CIGetPotentialCapabilities?$CJ?5unex@ 0000000180006bd8     libpopframe008.obj
 0002:00001c10       ??_C@_0CN@LKPEOJPO@?$CIAddCapabilities?$CJ?5unexpected?5er@ 0000000180006c10     libpopframe008.obj
 0002:00001c40       ??_C@_0CN@BCCBOHCH@?$CIGetCapabilities?$CJ?5unexpected?5er@ 0000000180006c40     libpopframe008.obj
 0002:00001c70       ??_C@_0CG@MCCDAOGE@Warning?3?5PopFrame?5is?5not?5implem@ 0000000180006c70     libpopframe008.obj
 0002:00001c98       ??_C@_0CP@IMINGNLL@?$CISetEventCallbacks?$CJ?5unexpected?5@ 0000000180006c98     libpopframe008.obj
 0002:00001cc8       ??_C@_0DN@NCDMFLGJ@Warning?3?5Breakpoint?5or?5SingleSt@ 0000000180006cc8     libpopframe008.obj
 0002:00001d08       ??_C@_0CH@CDOJMNAO@JVMTI?5client?5was?5not?5properly?5l@ 0000000180006d08     libpopframe008.obj
 0002:00001d30       ??_C@_0CH@JAFIADKC@Cannot?5get?5class?5of?5the?5thread?5@ 0000000180006d30     libpopframe008.obj
 0002:00001d58       ??_C@_01CKDDGHAB@D@        0000000180006d58     libpopframe008.obj
 0002:00001d60       ??_C@_0CF@NHBBNJBF@Cannot?5get?5Method?5ID?5for?5method@ 0000000180006d60     libpopframe008.obj
 0002:00001d88       ??_C@_0CH@OFMILGEO@Cannot?5get?5Method?5ID?5for?5method@ 0000000180006d88     libpopframe008.obj
 0002:00001db0       ??_C@_0CL@GMOLCHIJ@?$CISetBreakpoint?$CJ?5unexpected?5erro@ 0000000180006db0     libpopframe008.obj
 0002:00001de0       ??_C@_0CM@NEGFNKGE@Failed?5to?5enable?5BREAKPOINT?5eve@ 0000000180006de0     libpopframe008.obj
 0002:00001e10       ??_C@_0DA@DGKNOIBM@Wrong?5number?5of?5poped?5frames?3?5?$CF@ 0000000180006e10     libpopframe008.obj
 0002:00001e50       ??_C@_1EC@JIJBPKFM@?$AAa?$AAp?$AAi?$AA?9?$AAm?$AAs?$AA?9?$AAw?$AAi?$AAn?$AA?9?$AAc?$AAo?$AAr?$AAe@ 0000000180006e50     MSVCRT:thread_safe_statics.obj
 0002:00001e98       ??_C@_1BK@MGMFAEKH@?$AAk?$AAe?$AAr?$AAn?$AAe?$AAl?$AA3?$AA2?$AA?4?$AAd?$AAl?$AAl@ 0000000180006e98     MSVCRT:thread_safe_statics.obj
 0002:00001eb8       ??_C@_0BJ@JEBJOJFJ@SleepConditionVariableCS@ 0000000180006eb8     MSVCRT:thread_safe_statics.obj
 0002:00001ed8       ??_C@_0BJ@PGPPEPCC@WakeAllConditionVariable@ 0000000180006ed8     MSVCRT:thread_safe_statics.obj
 0002:00001ef8       _pDefaultRawDllMain        0000000180006ef8     MSVCRT:dll_dllmain.obj
 0002:00001ef8       _pRawDllMain               0000000180006ef8     MSVCRT:dll_dllmain.obj
 0002:00001f00       __xmm@ffffffffffffffffffffffffffffffff 0000000180006f00     MSVCRT:utility.obj
 0002:00001f10       _load_config_used          0000000180006f10     MSVCRT:loadcfg.obj
 0002:00002100       _tls_used                  0000000180007100     MSVCRT:tlssup.obj
 0002:00002128       __volatile_metadata        0000000180007128     <linker-defined>
 0002:000024f0       __rtc_iaa                  00000001800074f0     MSVCRT:initsect.obj
 0002:000024f8       __rtc_izz                  00000001800074f8     MSVCRT:initsect.obj
 0002:00002500       __rtc_taa                  0000000180007500     MSVCRT:initsect.obj
 0002:00002508       __rtc_tzz                  0000000180007508     MSVCRT:initsect.obj
 0002:00002510       _tls_start                 0000000180007510     MSVCRT:tlssup.obj
 0002:00002514       _Init_thread_epoch         0000000180007514     MSVCRT:thread_safe_statics.obj
 0002:00002518       _tls_end                   0000000180007518     MSVCRT:tlssup.obj
 0002:00002bf0       __IMPORT_DESCRIPTOR_KERNEL32 0000000180007bf0     kernel32:KERNEL32.dll
 0002:00002c04       __IMPORT_DESCRIPTOR_VCRUNTIME140 0000000180007c04     vcruntime:VCRUNTIME140.dll
 0002:00002c18       __IMPORT_DESCRIPTOR_api-ms-win-crt-runtime-l1-1-0 0000000180007c18     ucrt:api-ms-win-crt-runtime-l1-1-0.dll
 0002:00002c2c       __IMPORT_DESCRIPTOR_api-ms-win-crt-stdio-l1-1-0 0000000180007c2c     ucrt:api-ms-win-crt-stdio-l1-1-0.dll
 0002:00002c40       __IMPORT_DESCRIPTOR_api-ms-win-crt-string-l1-1-0 0000000180007c40     ucrt:api-ms-win-crt-string-l1-1-0.dll
 0002:00002c54       __NULL_IMPORT_DESCRIPTOR   0000000180007c54     kernel32:KERNEL32.dll
 0003:000000b0       _Init_global_epoch         00000001800090b0     MSVCRT:thread_safe_statics.obj
 0003:000000c0       __security_cookie          00000001800090c0     MSVCRT:gs_cookie.obj
 0003:000000c8       __security_cookie_complement 00000001800090c8     MSVCRT:gs_cookie.obj
 0003:000000d0       __scrt_native_dllmain_reason 00000001800090d0     MSVCRT:utility.obj
 0003:000000d8       __isa_available            00000001800090d8     MSVCRT:cpu_disp.obj
 0003:000000dc       __isa_enabled              00000001800090dc     MSVCRT:cpu_disp.obj
 0003:000000e0       __memset_fast_string_threshold 00000001800090e0     MSVCRT:cpu_disp.obj
 0003:000000e8       __memset_nt_threshold      00000001800090e8     MSVCRT:cpu_disp.obj
 0003:000000f0       __scrt_ucrt_dll_is_in_use  00000001800090f0     MSVCRT:ucrt_stubs.obj
 0003:00000100       g_wrongHeapCallbacks       0000000180009100     libpopframe008.obj
 0003:00000180       g_szTagInfo                0000000180009180     libpopframe008.obj
 0003:000020c0       g_tagFlags                 000000018000b0c0     libpopframe008.obj
 0003:000024a8       g_refsToVerifyCnt          000000018000b4a8     libpopframe008.obj
 0003:000024ac       g_fakeUserData             000000018000b4ac     libpopframe008.obj
 0003:000024b0       g_tagVisitCount            000000018000b4b0     libpopframe008.obj
 0003:00003450       g_refsToVerify             000000018000c450     libpopframe008.obj
 0003:0001ab50       g_userDataError            0000000180023b50     libpopframe008.obj
 0003:0001ae50       ?_OptionsStorage@?1??__local_stdio_printf_options@@9@4_KA 0000000180023e50     libpopframe008.obj
 0003:0001b418       _tls_index                 0000000180024418     MSVCRT:tlssup.obj
 0003:0001b420       __scrt_current_native_startup_state 0000000180024420     MSVCRT:utility.obj
 0003:0001b428       __scrt_native_startup_lock 0000000180024428     MSVCRT:utility.obj
 0003:0001b468       __scrt_debugger_hook_flag  0000000180024468     MSVCRT:utility_desktop.obj
 0003:0001b470       ?__type_info_root_node@@3U__type_info_node@@A 0000000180024470     MSVCRT:tncleanup.obj
 0003:0001b480       ?_OptionsStorage@?1??__local_stdio_scanf_options@@9@4_KA 0000000180024480     MSVCRT:default_local_stdio_options.obj
 0003:0001b488       __favor                    0000000180024488     MSVCRT:cpu_disp.obj
 0003:0001b490       __dyn_tls_init_callback    0000000180024490     <common>

 entry point at        0001:00002710

 Static symbols

 0000:fffd9000       .debug$S                   0000000180000000     popframe008.exp
 0000:fffd9000       .debug$S                   0000000180000000     vcruntime:VCRUNTIME140.dll
 0000:fffd9000       .debug$S                   0000000180000000     vcruntime:VCRUNTIME140.dll
 0000:fffd9000       .debug$S                   0000000180000000     vcruntime:VCRUNTIME140.dll
 0000:fffd9000       .debug$S                   0000000180000000     vcruntime:VCRUNTIME140.dll
 0000:fffd9000       .debug$S                   0000000180000000     vcruntime:VCRUNTIME140.dll
 0000:fffd9000       .debug$S                   0000000180000000     vcruntime:VCRUNTIME140.dll
 0000:fffd9000       .debug$S                   0000000180000000     vcruntime:VCRUNTIME140.dll
 0000:fffd9000       .debug$S                   0000000180000000     ucrt:api-ms-win-crt-convert-l1-1-0.dll
 0002:ffffb000       .idata$6                   0000000180000000     ucrt:api-ms-win-crt-convert-l1-1-0.dll
 0000:fffd9000       .debug$S                   0000000180000000     ucrt:api-ms-win-crt-heap-l1-1-0.dll
 0000:fffd9000       .debug$S                   0000000180000000     ucrt:api-ms-win-crt-heap-l1-1-0.dll
 0000:fffd9000       .debug$S                   0000000180000000     ucrt:api-ms-win-crt-heap-l1-1-0.dll
 0000:fffd9000       .debug$S                   0000000180000000     ucrt:api-ms-win-crt-heap-l1-1-0.dll
 0002:ffffb000       .idata$6                   0000000180000000     ucrt:api-ms-win-crt-heap-l1-1-0.dll
 0000:fffd9000       .debug$S                   0000000180000000     ucrt:api-ms-win-crt-runtime-l1-1-0.dll
 0000:fffd9000       .debug$S                   0000000180000000     ucrt:api-ms-win-crt-runtime-l1-1-0.dll
 0000:fffd9000       .debug$S                   0000000180000000     ucrt:api-ms-win-crt-runtime-l1-1-0.dll
 0000:fffd9000       .debug$S                   0000000180000000     ucrt:api-ms-win-crt-runtime-l1-1-0.dll
 0000:fffd9000       .debug$S                   0000000180000000     ucrt:api-ms-win-crt-runtime-l1-1-0.dll
 0000:fffd9000       .debug$S                   0000000180000000     ucrt:api-ms-win-crt-runtime-l1-1-0.dll
 0000:fffd9000       .debug$S                   0000000180000000     ucrt:api-ms-win-crt-runtime-l1-1-0.dll
 0000:fffd9000       .debug$S                   0000000180000000     ucrt:api-ms-win-crt-runtime-l1-1-0.dll
 0000:fffd9000       .debug$S                   0000000180000000     ucrt:api-ms-win-crt-runtime-l1-1-0.dll
 0000:fffd9000       .debug$S                   0000000180000000     ucrt:api-ms-win-crt-runtime-l1-1-0.dll
 0000:fffd9000       .debug$S                   0000000180000000     ucrt:api-ms-win-crt-runtime-l1-1-0.dll
 0000:fffd9000       .debug$S                   0000000180000000     ucrt:api-ms-win-crt-runtime-l1-1-0.dll
 0000:fffd9000       .debug$S                   0000000180000000     ucrt:api-ms-win-crt-runtime-l1-1-0.dll
 0000:fffd9000       .debug$S                   0000000180000000     ucrt:api-ms-win-crt-runtime-l1-1-0.dll
 0000:fffd9000       .debug$S                   0000000180000000     ucrt:api-ms-win-crt-runtime-l1-1-0.dll
 0000:fffd9000       .debug$S                   0000000180000000     ucrt:api-ms-win-crt-runtime-l1-1-0.dll
 0000:fffd9000       .debug$S                   0000000180000000     ucrt:api-ms-win-crt-stdio-l1-1-0.dll
 0000:fffd9000       .debug$S                   0000000180000000     ucrt:api-ms-win-crt-stdio-l1-1-0.dll
 0000:fffd9000       .debug$S                   0000000180000000     ucrt:api-ms-win-crt-stdio-l1-1-0.dll
 0000:fffd9000       .debug$S                   0000000180000000     ucrt:api-ms-win-crt-stdio-l1-1-0.dll
 0000:fffd9000       .debug$S                   0000000180000000     ucrt:api-ms-win-crt-stdio-l1-1-0.dll
 0000:fffd9000       .debug$S                   0000000180000000     ucrt:api-ms-win-crt-stdio-l1-1-0.dll
 0000:fffd9000       .debug$S                   0000000180000000     ucrt:api-ms-win-crt-stdio-l1-1-0.dll
 0000:fffd9000       .debug$S                   0000000180000000     ucrt:api-ms-win-crt-stdio-l1-1-0.dll
 0000:fffd9000       .debug$S                   0000000180000000     ucrt:api-ms-win-crt-stdio-l1-1-0.dll
 0000:fffd9000       .debug$S                   0000000180000000     ucrt:api-ms-win-crt-stdio-l1-1-0.dll
 0000:fffd9000       .debug$S                   0000000180000000     ucrt:api-ms-win-crt-string-l1-1-0.dll
 0000:fffd9000       .debug$S                   0000000180000000     ucrt:api-ms-win-crt-string-l1-1-0.dll
 0000:fffd9000       .debug$S                   0000000180000000     ucrt:api-ms-win-crt-string-l1-1-0.dll
 0000:fffd9000       .debug$S                   0000000180000000     ucrt:api-ms-win-crt-string-l1-1-0.dll
 0000:fffd9000       .debug$S                   0000000180000000     ucrt:api-ms-win-crt-string-l1-1-0.dll
 0000:fffd9000       .debug$S                   0000000180000000     ucrt:api-ms-win-crt-string-l1-1-0.dll
 0000:fffd9000       .debug$S                   0000000180000000     ucrt:api-ms-win-crt-string-l1-1-0.dll
 0000:fffd9000       .debug$S                   0000000180000000     ucrt:api-ms-win-crt-string-l1-1-0.dll
 0000:fffd9000       .debug$S                   0000000180000000     kernel32:KERNEL32.dll
 0000:fffd9000       .debug$S                   0000000180000000     kernel32:KERNEL32.dll
 0000:fffd9000       .debug$S                   0000000180000000     kernel32:KERNEL32.dll
 0000:fffd9000       .debug$S                   0000000180000000     kernel32:KERNEL32.dll
 0000:fffd9000       .debug$S                   0000000180000000     kernel32:KERNEL32.dll
 0000:fffd9000       .debug$S                   0000000180000000     kernel32:KERNEL32.dll
 0000:fffd9000       .debug$S                   0000000180000000     kernel32:KERNEL32.dll
 0000:fffd9000       .debug$S                   0000000180000000     kernel32:KERNEL32.dll
 0000:fffd9000       .debug$S                   0000000180000000     kernel32:KERNEL32.dll
 0000:fffd9000       .debug$S                   0000000180000000     kernel32:KERNEL32.dll
 0000:fffd9000       .debug$S                   0000000180000000     kernel32:KERNEL32.dll
 0000:fffd9000       .debug$S                   0000000180000000     kernel32:KERNEL32.dll
 0000:fffd9000       .debug$S                   0000000180000000     kernel32:KERNEL32.dll
 0000:fffd9000       .debug$S                   0000000180000000     kernel32:KERNEL32.dll
 0000:fffd9000       .debug$S                   0000000180000000     kernel32:KERNEL32.dll
 0000:fffd9000       .debug$S                   0000000180000000     kernel32:KERNEL32.dll
 0000:fffd9000       .debug$S                   0000000180000000     kernel32:KERNEL32.dll
 0000:fffd9000       .debug$S                   0000000180000000     kernel32:KERNEL32.dll
 0000:fffd9000       .debug$S                   0000000180000000     kernel32:KERNEL32.dll
 0000:fffd9000       .debug$S                   0000000180000000     kernel32:KERNEL32.dll
 0000:fffd9000       .debug$S                   0000000180000000     kernel32:KERNEL32.dll
 0000:fffd9000       .debug$S                   0000000180000000     kernel32:KERNEL32.dll
 0000:fffd9000       .debug$S                   0000000180000000     kernel32:KERNEL32.dll
 0000:fffd9000       .debug$S                   0000000180000000     kernel32:KERNEL32.dll
 0000:fffd9000       .debug$S                   0000000180000000     kernel32:KERNEL32.dll
 0000:fffd9000       .debug$S                   0000000180000000     kernel32:KERNEL32.dll
 0000:fffd9000       .debug$S                   0000000180000000     kernel32:KERNEL32.dll
 0000:fffd9000       .debug$S                   0000000180000000     kernel32:KERNEL32.dll
 0001:0000114c       addRefToVerify             000000018000214c f   libpopframe008.obj
 0001:000011c0       agentThreadWrapper         00000001800021c0 f   libpopframe008.obj
 0001:000015f8       file_basename              00000001800025f8 f   libpopframe008.obj
 0001:00001c20       startAgentThreadWrapper    0000000180002c20 f   libpopframe008.obj
 0001:00001f4c       syncDebuggeeStatus         0000000180002f4c f   libpopframe008.obj
 0001:000021d4       capture_previous_context   00000001800031d4 f   MSVCRT:gs_report.obj
 0001:00002248       ?__scrt_initialize_thread_safe_statics@@YAHXZ 0000000180003248 f   MSVCRT:thread_safe_statics.obj
 0001:00002318       ?__scrt_uninitialize_thread_safe_statics@@YAXXZ 0000000180003318 f   MSVCRT:thread_safe_statics.obj
 0001:000023c0       $$000000                   00000001800033c0     MSVCRT:amdsecgs.obj
 0001:000023f0       ?dllmain_crt_dispatch@@YAHQEAUHINSTANCE__@@KQEAX@Z 00000001800033f0 f   MSVCRT:dll_dllmain.obj
 0001:00002440       ?dllmain_crt_process_attach@@YAHQEAUHINSTANCE__@@QEAX@Z 0000000180003440 f   MSVCRT:dll_dllmain.obj
 0001:00002558       ?dllmain_crt_process_detach@@YAH_N@Z 0000000180003558 f   MSVCRT:dll_dllmain.obj
 0001:000025dc       ?dllmain_dispatch@@YAHQEAUHINSTANCE__@@KQEAX@Z 00000001800035dc f   MSVCRT:dll_dllmain.obj
 0001:00002ff0       $$000000                   0000000180003ff0     MSVCRT:guard_dispatch.obj
 0001:00003010       $$000000                   0000000180004010     MSVCRT:guard_xfg_dispatch.obj
 0001:00003026       ?fin$0@?0??dllmain_crt_process_attach@@YAHQEAUHINSTANCE__@@QEAX@Z@4HA 0000000180004026 f   MSVCRT:dll_dllmain.obj
 0001:0000303d       ?fin$0@?0??dllmain_crt_process_detach@@YAH_N@Z@4HA 000000018000403d f   MSVCRT:dll_dllmain.obj
 0001:00003056       ?fin$1@?0??dllmain_crt_process_detach@@YAH_N@Z@4HA 0000000180004056 f   MSVCRT:dll_dllmain.obj
 0001:0000306a       ?filt$0@?0??dllmain_dispatch@@YAHQEAUHINSTANCE__@@KQEAX@Z@4HA 000000018000406a f   MSVCRT:dll_dllmain.obj
 0001:000030a0       __scrt_is_nonwritable_in_current_image$filt$0 00000001800040a0 f   MSVCRT:utility.obj
 0002:000001e8       ?__scrt_initialize_tss_var@@3P6AHXZEA 00000001800051e8     MSVCRT:thread_safe_statics.obj
 0002:00000310       ?opcLengths@@3QBEB         0000000180005310     libpopframe008.obj
 0002:00001e40       GS_ExceptionPointers       0000000180006e40     MSVCRT:gs_report.obj
 0002:00002520       $unwind$fprintf            0000000180007520     libpopframe008.obj
 0002:0000252c       $unwind$printf             000000018000752c     libpopframe008.obj
 0002:00002538       $unwind$?NewObject@JNIEnv_@@QEAAPEAV_jobject@@PEAV_jclass@@PEAU_jmethodID@@ZZ 0000000180007538     libpopframe008.obj
 0002:00002538       $unwind$nsk_lcomplain      0000000180007538     libpopframe008.obj
 0002:00002538       $unwind$nsk_ldisplay       0000000180007538     libpopframe008.obj
 0002:00002540       $unwind$Java_nsk_jvmti_PopFrame_popframe008_getReady 0000000180007540     libpopframe008.obj
 0002:00002540       $unwind$nsk_lvdisplay      0000000180007540     libpopframe008.obj
 0002:00002540       $unwind$_RTC_Initialize    0000000180007540     MSVCRT:initsect.obj
 0002:00002540       $unwind$_RTC_Terminate     0000000180007540     MSVCRT:initsect.obj
 0002:00002540       $unwind$?__scrt_initialize_thread_safe_statics@@YAHXZ 0000000180007540     MSVCRT:thread_safe_statics.obj
 0002:0000254c       $unwind$nsk_lvcomplain     000000018000754c     libpopframe008.obj
 0002:00002564       $unwind$nsk_ltrace         0000000180007564     libpopframe008.obj
 0002:00002564       $unwind$__report_gsfailure 0000000180007564     MSVCRT:gs_report.obj
 0002:0000256c       $unwind$nsk_lvtrace        000000018000756c     libpopframe008.obj
 0002:0000256c       $unwind$__raise_securityfailure 000000018000756c     MSVCRT:gs_report.obj
 0002:0000256c       $unwind$__scrt_initialize_crt 000000018000756c     MSVCRT:utility.obj
 0002:0000256c       $unwind$__scrt_initialize_onexit_tables 000000018000756c     MSVCRT:utility.obj
 0002:0000256c       $unwind$__scrt_release_startup_lock 000000018000756c     MSVCRT:utility.obj
 0002:0000256c       $unwind$__scrt_uninitialize_crt 000000018000756c     MSVCRT:utility.obj
 0002:0000256c       $unwind$_onexit            000000018000756c     MSVCRT:utility.obj
 0002:00002574       $unwind$nsk_lverify        0000000180007574     libpopframe008.obj
 0002:00002584       $unwind$nsk_vprintf        0000000180007584     libpopframe008.obj
 0002:00002594       $unwind$nsk_printf         0000000180007594     libpopframe008.obj
 0002:0000259c       $unwind$?nsk_jni_lverify@@YAHHPEAUJNIEnv_@@HQEBDH1ZZ 000000018000759c     libpopframe008.obj
 0002:000025b0       $unwind$?nsk_jni_check_exception@@YAHPEAUJNIEnv_@@QEBDH@Z 00000001800075b0     libpopframe008.obj
 0002:000025cc       $unwind$Java_nsk_jvmti_PopFrame_popframe008_getRes 00000001800075cc     libpopframe008.obj
 0002:000025cc       $unwind$Java_nsk_jvmti_unit_FollowReferences_FollowRefObjects_resetTags 00000001800075cc     libpopframe008.obj
 0002:000025cc       $unwind$addRefToVerify     00000001800075cc     libpopframe008.obj
 0002:000025cc       $unwind$nsk_jvmti_resetAgentData 00000001800075cc     libpopframe008.obj
 0002:000025cc       $unwind$__scrt_initialize_default_local_stdio_options 00000001800075cc     MSVCRT:default_local_stdio_options.obj
 0002:000025cc       $unwind$?dllmain_crt_dispatch@@YAHQEAUHINSTANCE__@@KQEAX@Z 00000001800075cc     MSVCRT:dll_dllmain.obj
 0002:000025cc       $unwind$DllMain            00000001800075cc     MSVCRT:dll_dllmain_stub.obj
 0002:000025cc       $unwind$__GSHandlerCheck   00000001800075cc     MSVCRT:gshandler.obj
 0002:000025cc       $unwind$?__scrt_uninitialize_thread_safe_statics@@YAXXZ 00000001800075cc     MSVCRT:thread_safe_statics.obj
 0002:000025cc       $unwind$__scrt_acquire_startup_lock 00000001800075cc     MSVCRT:utility.obj
 0002:000025cc       $unwind$__scrt_dllmain_after_initialize_c 00000001800075cc     MSVCRT:utility.obj
 0002:000025cc       $unwind$__scrt_dllmain_before_initialize_c 00000001800075cc     MSVCRT:utility.obj
 0002:000025cc       $unwind$__scrt_dllmain_crt_thread_attach 00000001800075cc     MSVCRT:utility.obj
 0002:000025cc       $unwind$__scrt_dllmain_crt_thread_detach 00000001800075cc     MSVCRT:utility.obj
 0002:000025cc       $unwind$__scrt_dllmain_uninitialize_c 00000001800075cc     MSVCRT:utility.obj
 0002:000025cc       $unwind$__scrt_dllmain_uninitialize_critical 00000001800075cc     MSVCRT:utility.obj
 0002:000025cc       $unwind$atexit             00000001800075cc     MSVCRT:utility.obj
 0002:000025d4       $unwind$nsk_jvmti_lverify  00000001800075d4     libpopframe008.obj
 0002:000025e8       $unwind$exitOnError        00000001800075e8     libpopframe008.obj
 0002:000025f8       $unwind$Java_nsk_share_jvmti_ArgumentHandler_getAgentOptionsString 00000001800075f8     libpopframe008.obj
 0002:0000260c       $unwind$Java_nsk_jvmti_unit_FollowReferences_FollowRefObjects_getTag 000000018000760c     libpopframe008.obj
 0002:0000260c       $unwind$Java_nsk_share_jvmti_DebugeeClass_checkStatus 000000018000760c     libpopframe008.obj
 0002:0000260c       $unwind$agentThreadWrapper 000000018000760c     libpopframe008.obj
 0002:0000261c       $unwind$startAgentThreadWrapper 000000018000761c     libpopframe008.obj
 0002:00002638       $unwind$syncDebuggeeStatus 0000000180007638     libpopframe008.obj
 0002:00002638       $unwind$__scrt_dllmain_exception_filter 0000000180007638     MSVCRT:utility.obj
 0002:0000264c       $unwind$Java_nsk_share_jvmti_DebugeeClass_resetAgentData 000000018000764c     libpopframe008.obj
 0002:00002654       $unwind$MA_checkStatus     0000000180007654     libpopframe008.obj
 0002:00002668       $unwind$Java_nsk_jvmti_unit_FollowReferences_FollowRefObjects_setTag 0000000180007668     libpopframe008.obj
 0002:00002680       $unwind$Java_nsk_jvmti_unit_FollowReferences_FollowRefObjects_addRefToVerify 0000000180007680     libpopframe008.obj
 0002:0000269c       $unwind$Agent_Initialize   000000018000769c     libpopframe008.obj
 0002:000026a8       $unwind$check              00000001800076a8     libpopframe008.obj
 0002:000026c0       $unwind$Breakpoint         00000001800076c0     libpopframe008.obj
 0002:000026c0       $unwind$SingleStep         00000001800076c0     libpopframe008.obj
 0002:000026c0       $unwind$_DllMainCRTStartup 00000001800076c0     MSVCRT:dll_dllmain.obj
 0002:000026d0       $unwind$capture_previous_context 00000001800076d0     MSVCRT:gs_report.obj
 0002:000026dc       $unwind$__GSHandlerCheckCommon 00000001800076dc     MSVCRT:gshandler.obj
 0002:000026e8       $xdatasym                  00000001800076e8     MSVCRT:amdsecgs.obj
 0002:000026ec       $unwind$?dllmain_crt_process_attach@@YAHQEAUHINSTANCE__@@QEAX@Z 00000001800076ec     MSVCRT:dll_dllmain.obj
 0002:00002728       $unwind$?fin$0@?0??dllmain_crt_process_attach@@YAHQEAUHINSTANCE__@@QEAX@Z@4HA 0000000180007728     MSVCRT:dll_dllmain.obj
 0002:00002728       $unwind$?fin$0@?0??dllmain_crt_process_detach@@YAH_N@Z@4HA 0000000180007728     MSVCRT:dll_dllmain.obj
 0002:00002728       $unwind$?fin$1@?0??dllmain_crt_process_detach@@YAH_N@Z@4HA 0000000180007728     MSVCRT:dll_dllmain.obj
 0002:00002730       $unwind$?dllmain_crt_process_detach@@YAH_N@Z 0000000180007730     MSVCRT:dll_dllmain.obj
 0002:00002784       $unwind$?dllmain_dispatch@@YAHQEAUHINSTANCE__@@KQEAX@Z 0000000180007784     MSVCRT:dll_dllmain.obj
 0002:000027ac       $unwind$?filt$0@?0??dllmain_dispatch@@YAHQEAUHINSTANCE__@@KQEAX@Z@4HA 00000001800077ac     MSVCRT:dll_dllmain.obj
 0002:000027b4       $unwind$__scrt_is_nonwritable_in_current_image 00000001800077b4     MSVCRT:utility.obj
 0002:000027d4       $unwind$__scrt_is_nonwritable_in_current_image$filt$0 00000001800077d4     MSVCRT:utility.obj
 0002:000027dc       $unwind$__scrt_fastfail    00000001800077dc     MSVCRT:utility_desktop.obj
 0002:000027ec       $unwind$__security_init_cookie 00000001800077ec     MSVCRT:gs_support.obj
 0002:000027f8       $unwind$__isa_available_init 00000001800077f8     MSVCRT:cpu_disp.obj
 0002:00002808       $xdatasym                  0000000180007808     MSVCRT:guard_dispatch.obj
 0002:00002810       $xdatasym                  0000000180007810     MSVCRT:guard_xfg_dispatch.obj
 0002:00002820       .edata                     0000000180007820     popframe008.exp
 0002:00002848       rgpv                       0000000180007848     popframe008.exp
 0002:00002888       rgszName                   0000000180007888     popframe008.exp
 0002:000028c8       rgwOrd                     00000001800078c8     popframe008.exp
 0002:000028e8       szName                     00000001800078e8     popframe008.exp
 0002:000028f8       $N00001                    00000001800078f8     popframe008.exp
 0002:00002907       $N00002                    0000000180007907     popframe008.exp
 0002:00002914       $N00003                    0000000180007914     popframe008.exp
 0002:00002941       $N00004                    0000000180007941     popframe008.exp
 0002:0000296c       $N00005                    000000018000796c     popframe008.exp
 0002:000029b1       $N00006                    00000001800079b1     popframe008.exp
 0002:000029ee       $N00007                    00000001800079ee     popframe008.exp
 0002:00002a36       $N00008                    0000000180007a36     popframe008.exp
 0002:00002a76       $N00009                    0000000180007a76     popframe008.exp
 0002:00002ab3       $N00010                    0000000180007ab3     popframe008.exp
 0002:00002aee       $N00011                    0000000180007aee     popframe008.exp
 0002:00002b1c       $N00012                    0000000180007b1c     popframe008.exp
 0002:00002b4d       $N00013                    0000000180007b4d     popframe008.exp
 0002:00002b7c       $N00014                    0000000180007b7c     popframe008.exp
 0002:00002bab       $N00015                    0000000180007bab     popframe008.exp
 0002:00002be0       $N00016                    0000000180007be0     popframe008.exp
 0002:00002fea       .idata$6                   0000000180007fea     kernel32:KERNEL32.dll
 0002:0000304e       .idata$6                   000000018000804e     vcruntime:VCRUNTIME140.dll
 0002:000031ba       .idata$6                   00000001800081ba     ucrt:api-ms-win-crt-runtime-l1-1-0.dll
 0002:000031dc       .idata$6                   00000001800081dc     ucrt:api-ms-win-crt-stdio-l1-1-0.dll
 0002:000031fc       .idata$6                   00000001800081fc     ucrt:api-ms-win-crt-string-l1-1-0.dll
 0003:00000000       ?codeAttributeName@@3PEBDEB 0000000180009000     libpopframe008.obj
 0003:00000008       ?lineNumberAttributeName@@3PEBDEB 0000000180009008     libpopframe008.obj
 0003:00000010       ?localVarAttributeName@@3PEBDEB 0000000180009010     libpopframe008.obj
 0003:00000018       ?localVarTypeAttributeName@@3PEBDEB 0000000180009018     libpopframe008.obj
 0003:00000020       ?stackMapAttributeName@@3PEBDEB 0000000180009020     libpopframe008.obj
 0003:00000028       ?callBytes@@3PAEA          0000000180009028     libpopframe008.obj
 0003:0000002c       ?allocBytes@@3PAEA         000000018000902c     libpopframe008.obj
 0003:00000030       frames                     0000000180009030     libpopframe008.obj
 0003:0001ab54       redefineAttempted          0000000180023b54     libpopframe008.obj
 0003:0001ab58       nsk_context                0000000180023b58     libpopframe008.obj
 0003:0001ab64       redefineSucceed            0000000180023b64     libpopframe008.obj
 0003:0001ab68       agentFailed                0000000180023b68     libpopframe008.obj
 0003:0001ab6c       currentAgentStatus         0000000180023b6c     libpopframe008.obj
 0003:0001ab70       context                    0000000180023b70     libpopframe008.obj
 0003:0001ac28       agentThread                0000000180023c28     libpopframe008.obj
 0003:0001ac30       agentThreadProc            0000000180023c30     libpopframe008.obj
 0003:0001ac38       agentThreadArg             0000000180023c38     libpopframe008.obj
 0003:0001ac40       agent_data                 0000000180023c40     libpopframe008.obj
 0003:0001ac50       jvmti_env                  0000000180023c50     libpopframe008.obj
 0003:0001ac58       jvm                        0000000180023c58     libpopframe008.obj
 0003:0001ac60       jni_env                    0000000180023c60     libpopframe008.obj
 0003:0001ac68       checkStatus_func           0000000180023c68     libpopframe008.obj
 0003:0001ac70       ?codeAttributeIndex@@3GA   0000000180023c70     libpopframe008.obj
 0003:0001ac72       printdump                  0000000180023c72     libpopframe008.obj
 0003:0001ac74       ?lineNumberAttributeIndex@@3GA 0000000180023c74     libpopframe008.obj
 0003:0001ac78       ?localVarAttributeIndex@@3GA 0000000180023c78     libpopframe008.obj
 0003:0001ac7c       ?localVarTypeAttributeIndex@@3GA 0000000180023c7c     libpopframe008.obj
 0003:0001ac80       ?stackMapAttributeIndex@@3GA 0000000180023c80     libpopframe008.obj
 0003:0001ac84       ?stackFrameOffset@@3GA     0000000180023c84     libpopframe008.obj
 0003:0001ac88       ?mode@@3HA                 0000000180023c88     libpopframe008.obj
 0003:0001ac8c       ?constantPoolSize@@3GA     0000000180023c8c     libpopframe008.obj
 0003:0001ac90       ?orig@@3PEBEEB             0000000180023c90     libpopframe008.obj
 0003:0001ac98       ?gen@@3PEAEEA              0000000180023c98     libpopframe008.obj
 0003:0001aca0       ?inputPos@@3PEAEEA         0000000180023ca0     libpopframe008.obj
 0003:0001aca8       ?endPos@@3PEBEEB           0000000180023ca8     libpopframe008.obj
 0003:0001acb0       ?genPos@@3PEAEEA           0000000180023cb0     libpopframe008.obj
 0003:0001acb8       ?markPos@@3PEAEEA          0000000180023cb8     libpopframe008.obj
 0003:0001acc0       ?constantPool@@3PEAPEADEA  0000000180023cc0     libpopframe008.obj
 0003:0001acc8       ?constantPoolCount@@3GA    0000000180023cc8     libpopframe008.obj
 0003:0001accc       ?zeroBytes@@3PAEA          0000000180023ccc     libpopframe008.obj
 0003:0001acd0       ?codeLength@@3IA           0000000180023cd0     libpopframe008.obj
 0003:0001acd4       result                     0000000180023cd4     libpopframe008.obj
 0003:0001acd8       ?map@@3PEAIEA              0000000180023cd8     libpopframe008.obj
 0003:0001ace0       ?widening@@3PEACEA         0000000180023ce0     libpopframe008.obj
 0003:0001ace8       jvmti                      0000000180023ce8     libpopframe008.obj
 0003:0001acf0       caps                       0000000180023cf0     libpopframe008.obj
 0003:0001ad00       callbacks                  0000000180023d00     libpopframe008.obj
 0003:0001ae38       midD                       0000000180023e38     libpopframe008.obj
 0003:0001ae40       midRun                     0000000180023e40     libpopframe008.obj
 0003:0001ae48       framesExpected             0000000180023e48     libpopframe008.obj
 0003:0001ae4c       framesCount                0000000180023e4c     libpopframe008.obj
 0003:0001ae60       GS_ExceptionRecord         0000000180023e60     MSVCRT:gs_report.obj
 0003:0001af00       GS_ContextRecord           0000000180023f00     MSVCRT:gs_report.obj
 0003:0001b3d0       ?g_tss_cv@@3U_RTL_CONDITION_VARIABLE@@A 00000001800243d0     MSVCRT:thread_safe_statics.obj
 0003:0001b3d8       ?g_tss_event@@3PEAXEA      00000001800243d8     MSVCRT:thread_safe_statics.obj
 0003:0001b3e0       ?g_tss_mutex@@3U_RTL_CRITICAL_SECTION@@A 00000001800243e0     MSVCRT:thread_safe_statics.obj
 0003:0001b408       ?g_sleep_condition_variable_cs@@3P6AHPEAU_RTL_CONDITION_VARIABLE@@PEAU_RTL_CRITICAL_SECTION@@K@ZEA 0000000180024408     MSVCRT:thread_safe_statics.obj
 0003:0001b410       ?g_wake_all_condition_variable@@3P6AXPEAU_RTL_CONDITION_VARIABLE@@@ZEA 0000000180024410     MSVCRT:thread_safe_statics.obj
 0003:0001b41c       ?__proc_attached@@3HA      000000018002441c     MSVCRT:dll_dllmain.obj
 0003:0001b430       ?is_initialized_as_dll@@3_NA 0000000180024430     MSVCRT:utility.obj
 0003:0001b431       ?module_local_atexit_table_initialized@@3_NA 0000000180024431     MSVCRT:utility.obj
 0003:0001b438       ?module_local_atexit_table@@3U_onexit_table_t@@A 0000000180024438     MSVCRT:utility.obj
 0003:0001b450       ?module_local_at_quick_exit_table@@3U_onexit_table_t@@A 0000000180024450     MSVCRT:utility.obj
